:1009AF002811214112224214244418486F035E1F5C
:0C09BF00333D7D077F3701020408102043
:10000E00751101E511D39510500D740A1209E67899
:10001E0011740126F650EC22754001754100E52160
:10002E00F45540B4000A0541E540C333F54080EE77
:10003E00754010E521F45540B4000EE5412403F55A
:10004E0041E540C333F54080EAE541B40A05754108
:10005E00FF8008E541B4090375410A054185412237
:01006E00226F
:10006F00754300E540C4540FF542754100E5426405
:10007F0000600FE5412416F541E541D4F5411542E5
:06008F0080EBE540540F78
:100095002543F542E542D4F542E5412542F541E5E2
:1000A50041D4F541E54154F0FF7E0074041209F690
:1000B500E541540FFC7D00ED420EEC420F8E448F5E
:1000C5004522852D32852C4012006FEFF52E852CAB
:1000D5004012006F8E2FE52DB40513852B401200BD
:0E00E5006FEFF530852B4012006F8E318011C9
:0100F3008587
:1000F4002A4012006FEFF530852A4012006F8E31CE
:1001040022754000E540D39403501FE540242EF8A7
:100114008642E5429009BB120A1BE5402433F8E409
:1001240093F67840740126F650DAE5329009BB1252
:100134000A1BE493F541E541C4540FF537E541FF4B
:100144007401FEEF0E2303DEFD54804533F533E5E1
:1001540041FF7403FEEF0E2303DEFD54804534F5A6
:1001640034E541FF7402FEEF0E2303DEFD548045A7
:1001740035F535E541FF7404FEEF0E2303DEFD542F
:10018400804536F536E52764006044E5285401B41B
:10019400003BE5276401601A7405C395272433F8EE
:1001A400860FEF5480FF7405C395272433F8A60FF8
:1001B400801BE533547FF533E534547FF534E5355E
:0D01C400547FF535E536547FF5367537006C
:1001D100801BA2015009E5285401B400028002806D
:1001E1000CE5335480F533E5345480F534229046E0
:1001F10002E4F0904603E4F022C200E522B40B0FC2
:10020100E527B40505752701800205270202BCE533
:1002110022B40C1DE527B40105752601800DE52DDD
:0E022100B409051201EF80037526027527004F
:01022F0002CC
:1002300002BCE5279006C4F8282873752603807C45
:1002400085222D7527028074E52DB40510E52275F1
:10025000F00AA4FEAFF0EE2530F52B800EE52275F6
:10026000F00AA4FEAFF0EE2530F52A752703804C86
:10027000E52DB40510E53175F00AA4FEAFF0EE25CA
:1002800022F52B800EE53175F00AA4FEAFF0EE25C5
:1002900022F52A7527048024E52275F00AA4FEAF12
:1002A000F0EE252EF52C7527058011E52F75F00A47
:0C02B000A4FEAFF0EE2522F52C7527010E
:1006C40002023B0202400202480202700202980245
:0206D40002AB77
:0402BC002275130094
:1002C000E510C4540FF512751100E5126400600FBB
:1002D000E5112416F511E511D4F511151280EBE5A1
:1002E00010540F2513F512E512D4F512E51125125D
:1002F000F511E511D4F511E51154F0FF7E007404F9
:100300001209F6E511540FFC7D00ED4206EC4207A0
:100310008E148F1522904600E4F0A3F0751700E5C7
:100320001764FF700302042E904600E0FFA3E0FE76
:1003300074002EF58274443FF583E0F517E51764E9
:10034000FF70030204257402BF000FD39E400BE52B
:1003500017C4540F2430F516800B8517101202BDF8
:07036000EE2430F516C299EE
:10036700851699A299B3500280F9904600E0FFA341
:10037700E0FE7402BF000ED39E400AE517540F2417
:1003870030F516800B8517101202BDEF2430F516D5
:10039700C299851699A299B3500280F9904600E058
:1003A700FFA3E0FE74196E4F7002801A74336E4F0C
:1003B70070028012904600E0FFA3E0FE744D6E4F7E
:1003C70070028002801AC29975990AA299B35002E5
:1003D70080F9C29975990DA299B3500280F9803EB0
:1003E700904600E0FFA3E0FE740152067F00740010
:1003F7006E4F602A904600E0FFA3E0FE0EBE0001AC
:100407000F74002EF58274443FF583E0FFEF64FF1D
:0C041700600CC29975992CA299B3500298
:0604230080F99046001272
:100429000A0402031F751801E518D394085020C265
:100439009975990AA299B3500280F9C29975990DD3
:10044900A299B3500280F97818740126F650D9227E
:10045900E5269006D6F828287375260002057E75CC
:10046900260002057EE52BB40009852B1C12096FB5
:0504790002056DC20147
:10047E00E52DB40033A201B35009E52AC394075009
:10048E00028002800F852B1C12096FE52CB46302CB
:10049E00052A80E1A201B3500C752A00752C007458
:1004AE001090F202F002056D904603E0904400F0C9
:1004BE00904602E0904401F074FF904402F0740202
:1004CE00904600F8E4F0E8A3F0E52A6407605C8546
:1004DE002B1C12096FE52CB46304052A804B904641
:0104EE00000D
:1004EF00E0FFA3E0FE74002EF58274443FF583E530
:1004FF002AF0904600120A04904600E0FFA3E0FEA7
:0D050F0074002EF58274443FF583E52CF056
:10051C00904600120A04904600E0FFA3E0FE74002F
:10052C002EF58274443FF58374FFF0809E752A008B
:10053C00752C00741090F202F0120315904602E034
:10054C0004F0904602E0D4904602F0904602E0B4EB
:10055C00000F904603E004F0904603E0D49046036D
:10056C00F0752600800C752C63852B1C12096F7599
:02057C00260057
:0C06D60002046202046802046E02057255
:07057E0022758CCA758AFF8B
:010585000570
:1005860024D202E5296400600215297401FFE525DD
:100596005407FEEF8E09120003F547E525C42354E0
:1005A6001FF546E5462433F8860FEF55476400608D
:1005B60004D2B38002C2B3D2B2E525B44B05752589
:1005C6000080020525C2B2E525B40008D2B3D2B236
:0E05D600C2B20528E5245407B4005E7546EF56
:1005E400E54664FE6055E546440FF590859047E581
:1005F40047540F640F6021E547652360088547234E
:100604007546FE8011E5476521600B854721120080
:1006140026D2007546FE8021E546FF7401FEEF0EEA
:100624000323DEFDF546E546B4FE0EE52364FF60D4
:09063400057523FF80037521FF09
:02063D0080A596
:10063F00E525B400061200C7120105227590FF755B
:10064F009850758DF5758BF5758920D28CD28E7576
:10065F00A882753F00E53FD39409500FE53F24333F
:10066F00F87600783F740126F650EA752700752258
:0F067F00007521FF7523FF752600C201752C0041
:01068E0075F6
:10068F002A00752B01752D011201EF7510FA12005A
:10069F000E748290F203F0748290F303F0748B90D7
:1006AF00F403F0A20050031201FAE5266400600380
:0506BF0012045980EE59
:1006E200751900E519640A6005A201B3400280444D
:1006F200E5199009AF120A1BE49390F302F075100A
:100702005012000E90F301E05410B40002D201E541
:1007120019B4000E90F301E0540F640A6002D20192
:10072200800C90F301E0540F65196002D2010519A3
:10073200052C80AF22752C00C201744090F202F0A9
:0A074200751A00E51AD39403500E57
:10074C007510FA12000E781A740126F650EB74200C
:10075C0090F202F0751A00E51AD39403500E75103E
:0A076C00FA12000E781A740126F646
:1007760050EB90F202E4F0751BFE751A00E51A6460
:10078600086005A201B34002802EE51B90F000F040
:1007960090F001E0651B6002D20190F402E0651B57
:1007A6006002D201051AE51BFF7401FEEF0E03235A
:1007B600DEFDF51B052C80C5751BFE751A00E51AB6
:1007C60064086005A201B340028024E51B90F00294
:0907D600F090F100E0651B6002E7
:1007DF00D201051AE51BFF7401FEEF0E0323DEFDA8
:1007EF00F51B052C80CF751BFE751A00E51A6408E2
:0407FF006005A201EE
:10080300B340028024E51B90F101F090F102E06512
:100813001B6002D201051AE51BFF7401FEEF0E03F4
:1008230023DEFDF51B052C80CF751BFE751A00E535
:100833001A64086005A201B340028024E51B90F20C
:1008430000F090F201E0651B6002D201051AE51B7E
:0E085300FF7401FEEF0E0323DEFDF51B052CE6
:1008610080CF751BFE751A00E51A64036005A201AD
:10087100B340028038E51BF490F202F074051209CE
:10088100E6E51BFF7402FEEF0E0323DEFDFF90F48D
:1008910001E044E36F6002D201051AE51BFF740118
:0608A100FEEF0E0323DE52
:1008A700FDF51B052C80BBA201B3504A743F90F4A1
:1008B70000F0741090F202F090F302E4F07510501B
:1008C70012000E751A00E51A64066005A201B3400E
:1008D700028023E51AC454F0451A90F300F075100E
:1008E7005012000E90F301E0541064006002D20130
:0208F700051AE0
:1008F900052C80D0A201B3501B741090F202F07441
:100909000290F400F090F3007401F07510321200B7
:100919000E1206E2A201B35035741090F202F0747F
:100929000290F400F090F3007401F0751064120065
:100939000E1206E2A201B3501590F4007401F0748E
:100949001090F300F075106412000E1206E2A20175
:06095900B35012752C637F
:0A095F0090F202E4F090F302E4F0DD
:1009690090F400E4F022E51CD394014003751C01C6
:10097900E51C9009A9F8282873748290F003F07493
:100989009990F103F0748290F203F0748290F3036A
:0F099900F0748B90F403F01207378003123F00C5
:0609A9000209820209A50B
:0109A800222C
:090A1B002582F5825002058322B8
:0D0A0400A3E004F07006120A11E004F022D5
:08000300098002C333D9FC227D
:0E09F600048007C3CF33CFCE33CED5E0F62238
:1009E600600D782B0209F0007830D8FED5E0F822A9
:03000B000209CB1C
:03000000020A24CD
:090A240075815875D00002064BE3
:0A0A11000582D582021583158222AA
:1009CB00C0E0C0F0C083C082C0D075D00812057FD4
:0B09DB00D0D0D082D083D0F0D0E0322A
:0054530158
